:020000040000FA
:04000000FA3060284A
:080008008612601C8616AE0092
:10001000030EAF008312051E14284008E000601C88
:10002000861660188612A214051D1828BC0B142809
:100030002830BC000F30A3008B100314851E031062
:0C004000E00C2F0E8300AE0E2E0E090007
:1000C000203084008001840A80300402031C6228EE
:1000D0002830BC008316FE3085055F308605FF3072
:1000E00087058312850186018701103083168E00F3
:1000F0008312703083168F0083120030031799002B
:100100000313003003179A000313003097000030E8
:100110009F00003083169F008312003003179E005B
:100120000313003003179F000313C73083168100A9
:10013000831230309000003092000030831694001B
:10014000831200309400A63083169800831200308A
:1001500083169B0083120030980033308316990079
:100160008312003083168C008312003083168D00BA
:10017000831210308B00B20BBB280130A400810128
:100180008E018F010B118B100B108C128C018D01C5
:100190008B1764000B19DD20871BD028851DC9280B
:1001A000EC20C92848085002031DDA285008871E91
:1001B0005009C0004808D00008000B11A40B08002B
:1001C0000430A400A3080319E8288613A303080039
:1001D00006098039860008000514EE28EF28F0286B
:1001E000F128F228F328F428F528F628F728F8282B
:1001F000F928FA28FB280608A0000708A100051026
:10020000211807291430A50703180C2913291430C5
:10021000A502031C10291329FF30A5004814132937
:10022000A50148101329A1181A291430A60703188C
:100230001F2926291430A602031C23292629FF3052
:10024000A600C8142629A601C810262921192D297F
:100250001430A7070318322939291430A702031CC8
:1002600036293929FF30A70048153929A701481137
:100270003929201A40291430A807031845294C2988
:100280001430A802031C49294C29FF30A800C815C6
:100290004C29A801C8114C29211A53291430A90747
:1002A000031858295F291430A902031C5C295F290F
:1002B000FF30A90048165F29A90148125F29201BB9
:1002C00066291430AA0703186B2972291430AA0270
:1002D000031C6F297229FF30AA00C8167229AA01CF
:1002E000C8127229211B79291430AB0703187E2903
:1002F00085291430AB02031C82298529FF30AB000D
:1003000048178529AB0148138529A1198C29143078
:10031000AC070318912998291430AC02031C9529C5
:100320009829FF30AC00C8179829AC01C813982948
:04033000D2200800CF
:084000000800000001000000AF
:02400E00CC03E1
:00000001FF
